:04000000E8EF04F031
:0800080000C004F001C005F086
:1000100002C006F0076A03C008F000016F00D4FFB9
:1000200009F06F00D8FF0AF06F00DCFF0BF0390118
:1000300093AF1EEF00F0A3BFC4EF00F0600027F005
:10004000F5FF60002BF0F6FF60002FF0F7FF04C013
:1000500000F005C001F006C002F0078E08C003F0F2
:100060001100BC9C9F0E006E002EFED700D0CEEF7C
:1000700000F02F0E006E002EFED700D01200BC8CB8
:100080001A0E006E002EFED70000000B006E4850C6
:10009000040B036E0050031002E0BC8C01D0BC9C2A
:1000A000E8DF000B006E4850020B036E0050031097
:1000B00002E0BC8C01D0BC9CDCDF000B006E485021
:1000C000010B036E0050031002E0BC8C01D0BC9CFD
:1000D000D0DF4750800B006E036A0050031002E02F
:1000E000BC8C01D0BC9CC5DF4750400B006E036A3E
:1000F0000050031002E0BC8C01D0BC9CBADF47501A
:10010000200B006E036A0050031002E0BC8C01D08B
:10011000BC9CAFDF4750100B006E036A0050031009
:1001200002E0BC8C01D0BC9CA4DF4750080B006EE1
:10013000036A0050031002E0BC8C01D0BC9C99DF24
:100140004750040B006E036A0050031002E0BC8CA1
:1001500001D0BC9C8EDF4750020B006E036A00503A
:10016000031002E0BC8C01D0BC9C83DF4750010B24
:10017000006E036A0050031002E0BC8C01D0BC9CEE
:1001800078DFBC8CAEEF01F00001B8A801D0B76AEF
:10019000070EB66E2150030801E363D7436A43504C
:1001A0000108D8A0C8D0435003E0010A05E008D0F8
:1001B000446ACBB2442A06D0446ACBB0442A02D067
:1001C000010E446E4452D8A486D0036A43502D0FCA
:1001D000E96E000E0320EA6EEF5209E0036A435015
:1001E0002F0FE96E000E0320EA6E010EEF6E036A18
:1001F00043502D0FE96E000E0320EA6EEF6A445261
:1002000022E1D8904334036A310FE96E000E0320D7
:10021000EA6E6F00B0FF46F0ED526F00BCFF45F094
:100220004550F40803E1462C01D00DD0D89043345A
:10023000036A310FE96E000E0320EA6E010EEE260E
:1002400001E3EF2A47D0445245E1D8904334036A92
:10025000310FE96E000E0320EA6E6F00B0FF46F02A
:10026000ED526F00BCFF45F04550F40833E1462CD9
:1002700031D0036A43502F0FE96E000E0320EA6E5F
:10028000010EEF6E036A4350350FE96E000E032036
:10029000EA6EEF2A036A4350350FE96E000E032021
:1002A000EA6EEF500A0809E2036A4350370FE96E1D
:1002B000000E0320EA6E010EEF6ED8904334036AFD
:1002C000310FE96E000E0320EA6E010EEC6EED5266
:1002D000C20EEF6E2ED0036A43502D0FE96E000E52
:1002E0000320EA6E010EEF6ED8904334036A310F9B
:1002F000E96E000E0320EA6EEC6AED52EF6A036AC3
:100300004350350F016E000E032203C046F0036A0E
:100310004350370FE96E000E0320EA6EEF6A000EBD
:1003200060001BF1EAFF600007F0E9FF6F00A3FF28
:10033000EFFF432A34D72150030811E3D89021342A
:10034000036A190FE96E000E0320EA6E6F00B0FF1A
:1003500048F0ED526F00BCFF47F091D6212A392AB0
:10036000D8B43A2A3950E80806E13A50030803E1C4
:10037000216A3A6A396A3901A39F00011EEF00F031
:10038000EA6A3E0EE96EEF500EE0140E016E006A4E
:10039000002EFED7012EFBD7BF0E006E002EFED71B
:1003A00000D0EF2EF2D71200BC8ABC88C49AC49841
:1003B0003FEF05F0BC8CC49C40EF05F03D6A6F0038
:1003C00048FF3EF0D29E3901E16BE06BE59DE59F71
:1003D000E581E351E59DE58F3EBED28E4F0801E0F9
:1003E0003D2A6F0048FF3EF0D29EE16B010EE06FA8
:1003F000E59DE59FE581E351E59DE58F3EBED28E0B
:100400004B0801E03D2A6F0048FF3EF0D29EE16BB1
:10041000020EE06FE59DE59FE581E351E59DE58FE7
:100420003EBED28E490801E03D2A6F0048FF3EF0F3
:10043000D29EE16B030EE06FE59DE59FE581E35100
:10044000E59DE58F3EBED28E520801E03D2A6F0049
:1004500048FF3EF0D29EE16B040EE06FE59DE59F04
:10046000E581E351E59DE58F3EBED28E410801E076
:100470003D2A6F0048FF3EF0D29EE16B050EE06F13
:10048000E59DE59FE581E351E59DE58F3EBED28E7A
:100490004B0801E03D2A6F0048FF3EF0D29EE16B21
:1004A000060EE06FE59DE59FE581E351E59DE58F53
:1004B0003EBED28E550801E03D2ACBB201D03D2A86
:1004C000CBB001D03D2A3DC001F0000146EF05F060
:1004D000D250006ED29E3901E16BE06B4F0EE36F9C
:1004E000E59DE59FE585550EE66FAA0EE66FE5836F
:1004F000E5B3FED7E595E59DE58F0050D212D250C9
:10050000006ED29EE16B010EE06F4B0EE36FE59D36
:10051000E59FE585550EE66FAA0EE66FE583E5B328
:10052000FED7E595E59DE58F0050D212D250006EC2
:10053000D29EE16B020EE06F490EE36FE59DE59FF1
:10054000E585550EE66FAA0EE66FE583E5B3FED7A7
:10055000E595E59DE58F0050D212D250006ED29EF7
:10056000E16B030EE06F520EE36FE59DE59FE585BD
:10057000550EE66FAA0EE66FE583E5B3FED7E59567
:10058000E59DE58F0050D212D250006ED29EE16BF5
:10059000040EE06F410EE36FE59DE59FE585550E86
:1005A000E66FAA0EE66FE583E5B3FED7E595E59D18
:1005B000E58F0050D212D250006ED29EE16B050E34
:1005C000E06F4B0EE36FE59DE59FE585550EE66F09
:1005D000AA0EE66FE583E5B3FED7E595E59DE58FC9
:1005E0000050D212D250006ED29EE16B060EE06F28
:1005F000550EE36FE59DE59FE585E66FAA0EE66F74
:10060000E583E5B3FED7E595E59DE58F0050D21271
:100610002C68D250006ED29EE16B0A0EE06F600033
:10062000B3F0E3F9E59DE59FE585550EE66FAA0E6B
:10063000E66FE583E5B3FED7E595E59DE58F0050D0
:10064000D212000149EF05F06F0048FF3DF0D29E45
:100650003901E16B0A0EE06FE59DE59FE581E3510D
:10066000E59DE58F3DBED28E2C6E00014AEF05F070
:10067000150E006E002EFED7BC98150E006E002ED3
:10068000FED7BC9A150E006E002EFED7ADEF03F01C
:10069000BC880A0E006E002EFED70000BC8A0A0E2F
:1006A000006E002EFED70000BC9A0A0E006E002ECF
:1006B000FED700001200BC980A0E006E002EFED776
:1006C0000000BC8A0A0E006E002EFED70000BC9A05
:1006D0000A0E006E002EFED70000120042AE02D0BD
:1006E000D7DF01D0E8DF42AC02D0D2DF01D0E3DFB8
:1006F00042AA02D0CDDF01D0DEDF42A802D0C8DF9F
:1007000001D0D9DF42A602D0C3DF01D0D4DF42A49A
:1007100002D0BEDF01D0CFDF42A202D0B9DF01D0CC
:10072000CADF42A002D0B4DF01D0C5DF1200150E2F
:10073000006E002EFED7BC98150E006E002EFED760
:10074000BC8A150E006E002EFED7BC88150E006EFA
:10075000002EFED7BAEF03F08BD73FC042F0BEDFCA
:1007600097DF40C042F0BADF93DF41C042F0B6DF0E
:100770008FDFDDD71200226A236A2CC024F0256A9D
:10078000266A2CC027F0286A296A2A682B6A3D6AE3
:100790003D50090811E3036A3D50220FE96E000E37
:1007A0000320EA6E6F00BCFF41F0800E3F6E3DC03B
:1007B00040F0D2DF3D2AECD74BEF05F040500F0B55
:1007C0001FE0010A20E0030A21E0010A22E0070AF3
:1007D00023E0010A24E0030A25E0010A26E00F0ACB
:1007E00027E0010A28E0030A29E0010A2AE0070AB3
:1007F0002BE0010A2CE0030A2DE0010A2EE030D0A4
:100800003F0E416E2DD0060E416E2AD05B0E416E1A
:1008100027D04F0E416E24D0660E416E21D06D0E52
:10082000416E1ED07D0E416E1BD0070E416E18D05A
:100830007F0E416E15D06F0E416E12D0770E416E55
:100840000FD07C0E416E0CD0390E416E09D05E0E79
:10085000416E06D0790E416E03D0730E416E00D00A
:1008600041C001F012004150016A405C03E240C007
:1008700000F00CD0006A080E426E4036003641503F
:10088000005CD8B0006E0136422EF7D71200400E41
:100890003D5C006ED89000303E6E3D50400810E147
:1008A0001A6A196A1C6A1B6A406A88DF015080094B
:1008B0001D6E1E6A406A82DF206A01C01FF082D06E
:1008C0003D3C0DD01A6A370E196E1C6A3E0E1B6E27
:1008D0001E6A780E1D6E206A790E1F6E73D03E5010
:1008E00009081BE31A6A196A1C6A400E1B6E3EC097
:1008F00040F064DF015080091D6E1E6A3DA007D0E4
:10090000050E406E5BDF206A01C01FF005D0406A13
:1009100055DF206A01C01FF055D03E5063082DE31B
:100920003EC040F00A0E416E9EDF00C03FF03EC068
:1009300040F00A0E416E97DF01C03EF01A6A400E89
:10094000196E3EC040F03ADF1C6A01C01BF03FC088
:1009500040F034DF015080091D6E1E6A3DA007D0B3
:10096000050E406E2BDF206A01C01FF005D0406AE3
:1009700025DF206A01C01FF025D0640E3E5E3EC018
:1009800040F00A0E416E6FDF00C03FF03EC040F005
:100990000A0E416E68DF01C03EF01A6A400E196E01
:1009A000010E406E0BDF1C6A01C01BF03EC040F020
:1009B00005DF1E6A01C01DF03FC040F0FFDE206A67
:1009C00001C01FF01C801E82030E2012216A12003B
:1009D0003901E58FE59DF86AD29A078EDE6BDB6BF5
:1009E000DD6B080EDF6F600ED96F216A3A6A396AD3
:1009F0003A01406B506B606B806B3E01BD6BBE6B10
:100A0000BF6BBC6BB96BBA6BBB6BB86B010E2D6E59
:100A10002E6E2F6A306A316A326A336A346A356AF6
:100A2000366A376A386A3901DE6BDB6BDD6B030EC1
:100A3000DF6F600ED96F0A0E3E6E0001A1DC390136
:100A4000DE6BDB6BDD6B050EDF6F600ED96F0A0EA0
:100A50003E6E000195DC3901DE6BDB6BDD6B080E51
:100A6000DF6F600ED96F020E3D6EC80E3E6E000144
:100A700087DC3D2E01D002D03901F7D795D49AD426
:100A8000C382C3803A015169000198D40152D8A4AD
:100A90001FD5DAD570D6800EB86E460EB96EB8A8DE
:100AA00001D0B76A070EB66E3901938FC00ED2120D
:100AB0002CC03DF00001EBDE2CC03CF02F5205E0D5
:100AC0002F6A2C50400801E02C06305205E0306AB5
:100AD0002C3C01D001D02C2A3C502C5C2BE0800E09
:100AE0003F6E020E406E2CC041F036DE800E3F6E2F
:100AF000050E406E2CC041F02FDED250006ED29E0B
:100B00003901E16B0A0EE06F6000B3F0E3F9E59D97
:100B1000E59FE585550EE66FAA0EE66FE583E5B322
:100B2000FED7E595E59DE58F0050D2122CC03DF033
:080B30000001ADDEC1D7030096
:020000040030CA
:0A0000008CFF36FF9FFFFFDFFEFFBD
:00000001FF
